:1000000012C017C016C015C014C013C012C011C052
:1000100010C00FC00EC00DC00CC00BC00AC009C07C
:1000200008C007C006C011241FBECFEDCDBF14D03D
:100030002DC0E6CF02C0000001970097E1F70895B8
:10004000009749F02FEF3FEF000021503109E1F711
:100050000197C1F70895089511BA81E087BBC09850
:1000600026E030E08FEF9FEF00000197E9F7215085
:100070003109C1F7C09A26E030E08FEF9FEF000012
:100080000197E9F721503109C1F7E9CFF894FFCF83
:00000001FF
